:020000040000FA
:020000001028C6
:040002000034003492
:08000800A000030E8312A10009
:1000100005084B200B10210E8300A00E200E0900B6
:10002000831285011430990083168E1C1A280E1C29
:1000300052200E148E14A730990002309F01123006
:100040008500003095008830810010309600FF2335
:10005000900083128B018B158B170130A500810155
:1000600005112508FF3C0B1181000515191FA50A74
:10007000191BA5032508333A0319A50325080319FD
:100080002514323CFF3C0B1D43280B118100051148
:100090000B1D4828312805110130A5005220051AF2
:1000A0004F2808000730A2002F30A3000330A4001F
:1000B000A20B5B28A30B5D28A40B58285F2860289F
:0400C00061280800AB
:02400E00C401EB
:00000001FF
